:100000000C940F020C9456020C9456020C94560257
:100010000C9456020C9456020C9456020C94560200
:100020000C9456020C9456020C946A0B0C943C0CE3
:100030000C9456020C9456020C9456020C945602E0
:100040000C9456020C94B0200C9456020C94560258
:100050000C9456020C94421A0C9456020C945602BC
:100060000C9456020C9456020C9456020C945602B0
:100070000C9456020C9456020C9456020C945602A0
:100080000C9456020C9456020C9456020C94560290
:100090000C9456020C9456020C9456020C94560280
:1000A0000C9456020C9456020C945602A90CCB0CDC
:1000B000BE0DCB0CBE0D100D330DBE0D880D9B0D6E
:1000C00085108510B410B410F71031113E133E1393
:1000D0004A113E133F123F1212133E133E132913CF
:1000E00023024C003900E100640000001E001400EF
:1000F00004001D714A0039001F001A0016001B730E
:100100004E002A0020000800070006744B002B0058
:1001100021001500090019004D006400220017009D
:100120000A00050000006574AE0001540000007F65
:100130000000E300AB000154000000770000E20083
:1001400023001C000B00110000002971240018007E
:100150000D0010005000E60025000C000E003600D7
:1001600051002800260012000F00370052002C001A
:1001700027001300330038004F0031002D002F00FE
:100180003400E50029000000010001000100010029
:10019000010000003A000100F700FB00010001002F
:1001A0003B00F400F200FA00FD00F5003C00F00016
:1001B000F100F900FE00F4003D00F500F300FC0042
:1001C000FF0001003E000100F800F6000000010001
:1001D0000100010000000100000001000100010019
:1001E00000000100000001003F0001000100B40018
:1001F000000001004000AA00AC00B60001000100B0
:100200004100A800AD00B5000100B7004200A90000
:10021000AE00B9000100B60043000100AB00B7001A
:100220000100010044004500010001000100000040
:1002300016034500720067006F0044006F007800ED
:10024000200045005A0000001603450072006700B8
:100250006F0044006F007800200045005A00000045
:100260000403090409026D00040100A0FA09040056
:10027000000103010100092111010001223F0007D3
:1002800005810308000A09040100010301020009B5
:100290002111010001224D000705820308000A090F
:1002A00004020001030000000921110100012236AF
:1002B000000705830308000A090403000103000086
:1002C00000092111010001223900070584031000F3
:1002D000011201100100000008EDFE0713010001EA
:1002E00002000105010906A101050719E029E7152A
:1002F0000025019508750181020508190129059558
:1003000005750191029501750391010507190029F1
:100310007715002501957875018102C005010980D6
:10032000A101850216010026B7001A01002AB700B4
:10033000751095018100C0050C0901A10185031606
:100340000100269C021A01002A9C02751095018169
:1003500000C005010902A1010901A1000509190157
:100360002905150025019505750181029501750383
:1003700081010501093009311581257F9502750834
:10038000810609381581257F950175088106050CC0
:100390000A38021581257F950175088106C0C005C0
:1003A000010906A101050719E029E71500250195B6
:1003B0000875018102950175088101050819012957
:1003C00005950575019102950175039101050719C0
:1003D0000029FF150025FF950675088100C0000063
:1003E000000000000000000000010204060A0F17D0
:1003F000202C3A4A5D71879DB3C7DAE9F5FCFFFC12
:10040000F5E9DAC7B39D87715D4A3A2C20170F0AC8
:10041000060402010000000000000000000011249A
:100420001FBECFEFDAE0DEBFCDBF04B603FE27C0AC
:100430008091ED019091EE01A091EF01B091F0015A
:100440008730904BA740B04BD1F41092ED01109241
:10045000EE011092EF011092F00114BE84B7877F75
:1004600084BF0FB6F894A89580916000886180934E
:100470006000109260000FBEE0E0FFE3099511E01C
:10048000A0E0B1E0E2E0F5E402C005900D92A433F3
:10049000B107D9F721E0A4E3B1E001C01D92AD3E60
:1004A000B207E1F70E94B1080C947F220C9400007F
:1004B00061110BC0FC018281882321F085EE0E942E
:1004C0001F0F03C085EE0E94E70F80E090E00895C3
:1004D00008956091B1017091B2018091B301909142
:1004E000B4010E946F1956985E9825982D98269809
:1004F0002E9827982F98813019F4269A2E9A0895CD
:1005000056985E9808950C94690256985E982598BE
:100510002D9826982E9827982F988FEF90E09093FB
:1005200089008093880090938B0080938A00909339
:100530008D0080938C00259A2D9A2FEF80E792E012
:10054000215080409040E1F700C00000269A2E9A8A
:100550002FEF80E792E0215080409040E1F700C00B
:100560000000279A2F9A2FEF80E792E021508040D9
:100570009040E1F700C0000025982D982FEF80E70C
:1005800092E0215080409040E1F700C000002698A2
:100590002E982FEF80E792E0215080409040E1F7C5
:1005A00000C0000027982F9856985E9825982D989F
:1005B00026982E9827982F98089589EA809380008E
:1005C00089E08093810024982C983F988AB18F7499
:1005D0008AB96E98479A8BB1806B8BB9769A0E94D4
:1005E00085020C94680280E28093000180913401BE
:1005F00081110EC00E94420381E0809334012FEFED
:1006000083ED90E3215080409040E1F700C000006E
:1006100080E40E9448038093000181112EC00E9453
:10062000720380930001811128C00E94720380939D
:100630000001811122C08FE30E94720380930001A8
:1006400081111BC00E946A0380E40E9448038093CA
:100650000001811112C08CE00E947203809300019E
:1006600081110BC00E94720380930001811105C0AB
:100670008FE30E947203809300010E946A038091BD
:10068000000108951092B9008AE08093B80008959F
:1006900094EA9093BC009091BC0097FFFCCF90919E
:1006A000B900987F983021F0903111F081E00895E1
:1006B0008093BB0084E88093BC008091BC0087FFDE
:1006C000FCCF8091B900887F883111F0803471F7B8
:1006D00080E0089584E98093BC008091BC0084FD93
:1006E000FCCF08958093BB0084E88093BC00809188
:1006F000BC0087FFFCCF9091B900987F81E09832D1
:1007000009F480E0089584E88093BC008091BC00E7
:1007100087FFFCCF8091BB0008958091000181117B
:1007200015C080E40E9448038093000181110CC031
:1007300082E10E94720380930001811105C08FEF56
:100740000E947203809300010E946A0384B1807F3B
:1007500084B985B1807F85B98AB1837F8AB98BB12D
:10076000837F8BB93E98469808950E94F302809348
:1007700000010E948D0380B38C7080BB81B3836FB6
:1007800081BBE4E4F1E0A6E3B1E011921D9281E0C7
:10079000E235F807D1F70C94DD029F92AF92BF9239
:1007A000CF92DF92EF92FF920F931F93CF93DF933D
:1007B00080910001882379F0809135018F5F8093CB
:1007C0003501811108C00E94F3028093000181115C
:1007D00002C00E94850286E3E82E81E0F82E8701A0
:1007E000C0E0D0E0BB24B39492E0A92ECC24C39403
:1007F000D12CC730D10500F580910001811164C072
:1008000080E40E94480380930001811112C082E1BC
:100810000E9472038093000181110BC0C6010C2E4F
:1008200001C0880F0A94EAF780950E9472038093B2
:1008300000010E946A0348C0CA30A1F028F4C83001
:1008400059F0C93061F005C0CC3089F070F0CD307E
:1008500089F0209A289810C0219A29980DC0229AD0
:100860002A980AC0239A2B9807C0529A01C0539A1B
:100870005B9802C03E9A4698E0EAEA95F1F78FB19C
:1008800081708B25799902C032E001C030E0832B62
:100890007C9902C034E001C030E0832B7D9902C016
:1008A00028E001C020E0822B7E9902C090E101C0C7
:1008B00090E0892B9FB19095991F9927991F929548
:1008C000990F907E892B0FC08091000181114AC041
:1008D00080E40E94480380930001882381F1912CD9
:1008E0000E946A03892DD8019C91981719F08C9366
:1008F000A09201010E948D0321960F5F1F4FCE3001
:10090000D10509F076CF80910101882369F18150EA
:1009100080930101882339F0EFE9FFE03197F1F787
:1009200000C0000021C0E4E4F1E0D7018D917D0119
:100930008193B4E4EB16B1E0FB06B9F715C083E18F
:100940000E947203809300018111C9CF81E40E944B
:100950004803809300018111C2CF0E948303982E27
:100960009094BECF80E0BFCF0E94830281E0DF91F0
:10097000CF911F910F91FF90EF90DF90CF90BF909C
:10098000AF909F900895E82FF0E0EC5BFE4F8081E0
:10099000089508958B3B910580F4883A910548F5B8
:1009A000853A9105D8F48430910508F0B2C00197DA
:1009B00009F06EC081E090E00895803E910508F452
:1009C00067C0883E910508F4A4C09C01205F3109EE
:1009D0002031310508F05CC090650895853A910595
:1009E00009F459C0863A910509F058C082E890E4AC
:1009F0000895883A910509F454C0893A910509F49B
:100A000053C08A3A910509F452C08B3A910509F412
:100A100051C08C3A910509F450C08D3A910509F402
:100A20004FC0803B910509F44EC08E3A910509F400
:100A30004DC08F3A910509F44CC0813B910509F4F2
:100A40004BC0823B910509F44AC0833B910509F4F0
:100A500049C0843B910509F448C0853B910509F4E0
:100A600047C0863B910509F446C0873B910509F4D0
:100A700045C0883B910509F444C0893B910509F4C0
:100A800043C08A3B910509F442C080E094E4089594
:100A900080E090E0089581E890E4089583E890E490
:100AA000089582EE94E4089589EE94E408958AEE20
:100AB00094E4089585EB94E4089586EB94E4089516
:100AC00087EB94E408958CEC94E408958DEC94E421
:100AD000089583E895E408958AE895E4089582E905
:100AE00095E4089584E995E4089581E296E40895F3
:100AF00083E296E4089584E296E4089585E296E41C
:100B0000089586E296E4089587E296E408958AE2DD
:100B100096E40895089524E5829FC0011124FC0104
:100B200026E0729FE00DF11D1124E60FF11DEE0F7E
:100B3000FF1FE052FF4F859194910895880F991FF0
:100B4000FC01E05AF040859194910895880F991F17
:100B5000FC01E052FF4F85919491089524E5829F16
:100B6000C0011124FC0146E0749FE00DF11D112429
:100B7000E60FF11DEE0FFF1FE052FF4F859194919C
:100B80009C013A9521154FE1340708F425C13F51E6
:100B90002115304120F49F700E94A60508959C0104
:100BA00030532115304118F49927906C0895811520
:100BB00020E5920769F40E9460134FEF84E39CE004
:100BC000415080409040E1F700C000000C94671A4B
:100BD000813020E5920731F48091CC0181608093CF
:100BE000CC0108959C0130552115304108F05CC0BE
:100BF000292F33272F70332721303105E9F4AC0139
:100C000064E0440F551F6A95E1F744275370BC0117
:100C10006370772702C0220F331F6A95E2F73C68A2
:100C2000242B352B73E0880F991F7A95E1F7807696
:100C30009927822B932B08952230310529F4982F80
:100C40008827816F906A089523303105A1F4AC01A3
:100C500033E0440F551F3A95E1F7407E577083709B
:100C6000992721E030E002C0220F331F8A95E2F776
:100C7000C9019C6816C02430310531F5AC0123E070
:100C8000440F551F2A95E1F7407E577083709927CE
:100C900021E030E002C0220F331F8A95E2F7C9013C
:100CA0009A68842B952B08959C013057211530416B
:100CB00018F49F70906208959C01305821153041BE
:100CC00018F49F70906A0895803E9105E0F4803C8E
:100CD000910558F58133910509F46FC048F48932C4
:100CE000910509F463C08A32910509F46DC072C0A0
:100CF00089339105E9F082389105D1F0853391056A
:100D000009F44DC067C0833E910581F138F4803EFF
:100D10009105B9F0823E9105D9F05CC0863E9105FF
:100D200061F1873E9105A1F155C00E949E0508958D
:100D30002091DE0120FD02C021FF4CC080EE90E03A
:100D400049C08091DE0180FFF9CF89E390E042C085
:100D50008091DE0182FF0EC08091DE0184FF03C01E
:100D600080E090E037C083EE90E034C08091DE01F7
:100D700082FFF2CF82EE90E02DC08091DE0183FFF2
:100D80000BC08091DE0184FDEBCF87EE90E022C0A6
:100D90008091DE0183FFF5CF86EE90E01BC080914D
:100DA000DE0185FF07C089E290E014C08091DE017A
:100DB00085FFF9CF85E390E00DC08091DE0186FFCD
:100DC00007C08AE290E006C08091DE0186FFF9CF7D
:100DD00081E390E00E94CA04089508958091620121
:100DE0000895CF93DF9300D01F92CDB7DEB79C015B
:100DF0008091E401843019F593E099833B832A8341
:100E00009093E9008FEF9091E800815095FD06C026
:100E100095ED9A95F1F700008111F5CF8091E800EA
:100E200085FF0DC040E050E063E070E0CE01019628
:100E30000E945E098091E8008E778093E8000F9011
:100E40000F900F90DF91CF910895CF93DF9300D053
:100E50001F92CDB7DEB72091E401243021F522E0C6
:100E600029839B838A8383E08093E9008FEF9091AD
:100E7000E800815095FD06C095ED9A95F1F70000C8
:100E80008111F5CF8091E80085FF0DC040E050E072
:100E900063E070E0CE0101960E945E098091E80057
:100EA0008E778093E8000F900F900F90DF91CF9195
:100EB00008959C018091E4018430F9F482E08093EC
:100EC000E9009FEF8091E800915085FD06C085ED17
:100ED0008A95F1F700009111F5CF8091E80085FF28
:100EE0000CC040E050E065E070E0C9010E945E097E
:100EF0008091E8008E778093E8000895CF93DF9388
:100F0000EC018091E401843009F046C090910C011D
:100F10009923D9F090910D019923B9F08093E900BC
:100F20008FEF9091E800815095FD06C095E19A956C
:100F3000F1F700008111F5CF8091E80085FF2CC00A
:100F400040E050E060E170E017C081E08093E9008C
:100F50008FEF9091E800815095FD06C095ED9A9530
:100F6000F1F700008111F5CF8091E80085FF14C0F2
:100F700040E050E068E070E0CE010E945E098091A0
:100F8000E8008E778093E80080E1FE01A2E5B1E001
:100F900001900D928A95E1F7DF91CF9108958091AC
:100FA000E301811109C00E94EF0A0E944C0B80915D
:100FB000E20084608093E20008951092E3010895B6
:100FC00008950C949D200E94FD190E94A3200E9468
:100FD000F70D0C94ED0642E061EC81E00E94680A96
:100FE00042E061EC82E00E94680A42E061EC83E04A
:100FF0000E94680A42E161EC84E00C94680A8091E6
:10100000E601833009F455C030F4813071F082304C
:1010100009F48EC008958A3009F47AC08B3009F43F
:1010200060C0893009F09CC020C08091E501813A00
:1010300009F096C08091E800877F8093E800809156
:10104000E9019091EA01892B21F460E182E591E0C8
:1010500003C060E080E090E070E00E94A909809108
:10106000E8008B778093E80008958091E501813254
:1010700009F076C08091E9019091EA01009719F09A
:10108000039709F06DC08091E800877F8093E800A6
:101090008091E80082FD05C08091E4018111F8CFC4
:1010A0005FC08091F100809362018091E8008B77AE
:1010B00053C08091E501813A09F052C08091E90165
:1010C0009091EA01892B09F04BC08091E800877F5D
:1010D0008093E8008091E80080FFFCCF80910C01B4
:1010E00036C08091E5018132D9F58091E901909176
:1010F000EA01892BA9F58091E800877F8093E800B9
:101100000E949D0A8091E70180930C010C9460136A
:101110008091E501813221F58091E800877F8093FD
:10112000E8000E949D0A8091E80180936301089580
:101130008091E501813AA1F48091E800877F809356
:10114000E8008091E80080FFFCCF809163018093EC
:10115000F1008091E8008E778093E8000C949D0A5E
:10116000089584B7877F84BF0FB6F894A8958091BF
:101170006000886180936000109260000FBE90E074
:1011800080E80FB6F89480936100909361000FBEE1
:101190000E94460E0E94EF0A0E944C0B8091E200D2
:1011A00084608093E20078940E94D70D0E94480EDC
:1011B00082E091E00E94F20D0E948B208091E40178
:1011C000853069F40E94BF198091E2018823B1F350
:1011D0000E94E919882391F30E944809EFCF0E94E9
:1011E0004E0EECCF292F332723303105C9F060F4A0
:1011F0002130310581F02230310509F041C08DE602
:1012000090E024E632E040C021323105E1F02232A4
:10121000310531F135C082E190E021ED32E034C09A
:1012200099278130910549F028F0029749F5E0E3CC
:10123000F2E005C0E0E6F2E002C0E8E4F2E084910A
:1012400090E09F0121C06430D8F4E62FF0E0EE0F6B
:10125000FF1FEE5DFE4F2081318189E090E014C0D8
:10126000643070F470E0FB01EE0FFF1FE65EFE4F8E
:1012700020813181FB01EA5EFE4F808190E004C055
:1012800080E090E020E030E0FA013183208308958F
:1012900080E189BD82E189BD09B400FEFDCF809166
:1012A000D8008F7D8093D8008091E0008260809389
:1012B000E0008091E00081FDFCCF0895CF92DF92A5
:1012C000EF92FF920F931F93CF93DF93EC018B016B
:1012D0006A010E94BC0A811133C0C114D10439F0E3
:1012E000F60180819181081B190BC80FD91FE12CD1
:1012F000F12C0115110519F18091E80085FD16C04A
:101300008091E8008E778093E800C114D10449F001
:10131000F60180819181E80EF91EF182E08285E07C
:101320000FC00E94BC0A882321F30AC089918093D0
:10133000F10001501109FFEFEF1AFF0ADACF80E048
:10134000DF91CF911F910F91FF90EF90DF90CF90A1
:1013500008952091EB013091EC012617370748F0F2
:101360006115710539F42091E8002E772093E8008B
:1013700001C0B901FC0120E06115710579F180918E
:10138000E4018823F1F18530F1F18091E80083FDDB
:101390003CC08091E80082FD2EC08091E80080FF73
:1013A000EBCF2091F3008091F20090E0922B611539
:1013B000710551F08830910538F421912093F100A6
:1013C000615071090196F3CF21E0089709F020E000
:1013D0008091E8008E778093E800CECF2111CFCFA7
:1013E0000AC08091E401882361F0853061F080912A
:1013F000E80083FD0AC08091E80082FFF2CF80E020
:10140000089582E0089583E0089581E00895209191
:10141000EB013091EC012617370748F06115710593
:1014200039F42091E8002E772093E80001C0B9013B
:10143000FC0120E06115710591F18091E4018823A0
:1014400009F440C0853009F43FC08091E80083FD75
:101450003DC08091E80082FD2FC08091E80080FFB0
:10146000E9CF2091F3008091F20090E0922B61157A
:10147000710559F08830910540F424912093F100D2
:101480003196615071090196F2CF21E0089709F079
:1014900020E08091E8008E778093E800CBCF211187
:1014A000CCCF0AC08091E401882361F0853061F0DF
:1014B0008091E80083FD0AC08091E80082FFF2CFAE
:1014C00080E0089582E0089583E0089581E0089522
:1014D000982F973068F59093E900981739F070913C
:1014E000EC002091ED005091F00003C0242F762FE6
:1014F00050E021FD02C09F5FECCF3091EB003E7FBA
:101500003093EB003091ED003D7F3093ED00309152
:10151000EB0031603093EB007093EC002093ED0012
:101520005093F0002091EE0027FDE5CF80E0089574
:101530008F708093E90081E008958091E50187FF35
:1015400011C08091E80082FD05C08091E401811105
:10155000F8CF11C08091E8008B770BC08091E40137
:10156000882349F08091E80080FFF8CF8091E8005F
:101570008E778093E80008952091E4003091E50093
:1015800095E64091EC00842F817040FF23C080914C
:10159000E80080FD1DC08091E401882399F085302A
:1015A00099F08091EB0085FD11C04091E4005091CD
:1015B000E5002417350729F3915011F09A01E1CF86
:1015C00084E0089582E0089583E0089581E008951D
:1015D00080E008954091E80042FFDDCF08950E9429
:1015E0005D0B0E94650BE0EEF0E0808181608083FE
:1015F000E8EDF0E080818F77808319BCA7EDB0E043
:101600008C918E7F8C9380818F7E80831092E301FA
:1016100008950F931F93CF93DF930E945D0B0E9459
:10162000650BC8EDD0E088818F77888388818068DA
:10163000888388818F7D888319BC1092E401109281
:10164000E0011092E2011092E10100EE10E0F801D9
:1016500080818B7F808388818160888342E060E025
:1016600080E00E94680AE1EEF0E080818E7F808356
:10167000E2EEF0E0808181608083808188608083F9
:10168000F80180818E7F8083888180618883DF91EB
:10169000CF911F910F910895E8EDF0E080818F7E4A
:1016A0008083E7EDF0E080818160808384E082BF09
:1016B00081E08093E3010C94090BE8EDF0E0808178
:1016C0008E7F80831092E20008951092DA001092CB
:1016D000E10008951F920F920FB60F9211242F93DD
:1016E0003F934F935F936F937F938F939F93AF93AA
:1016F000BF93EF93FF938091E10082FF0BC0809135
:10170000E20082FF07C08091E1008B7F8093E100BF
:101710000E94D60D8091DA0080FF1FC08091D80012
:1017200080FF1BC08091DA008E7F8093DA00809169
:10173000D90080FF0DC080E189BD82E189BD09B477
:1017400000FEFDCF81E08093E4010E94CF0705C039
:1017500019BC1092E4010E94DD078091E10080FF36
:1017600019C08091E20080FF15C08091E2008E7F59
:101770008093E2008091E20080618093E20080919A
:10178000D80080628093D80019BC85E08093E40182
:101790000E94E1078091E10084FF30C08091E20067
:1017A00084FF2CC080E189BD82E189BD09B400FEBF
:1017B000FDCF8091D8008F7D8093D8008091E1008B
:1017C0008F7E8093E1008091E2008F7E8093E20023
:1017D0008091E20081608093E2008091E0018823A3
:1017E00011F084E007C08091E30087FD02C081E032
:1017F00001C083E08093E4010E94E3078091E1004F
:1018000083FF29C08091E20083FF25C08091E10021
:10181000877F8093E10082E08093E4011092E001F1
:101820008091E1008E7F8093E1008091E2008E7FC5
:101830008093E2008091E20080618093E20042E0C8
:1018400060E080E00E94680A8091F00088608093E8
:10185000F0000E94E007FF91EF91BF91AF919F913F
:101860008F917F916F915F914F913F912F910F9049
:101870000FBE0F901F9018951F920F920FB60F92E8
:1018800011242F933F934F935F936F937F938F9385
:101890009F93AF93BF93CF93DF93EF93FF93C09149
:1018A000E900CF708091EC00D82FD17080FDD0E896
:1018B0001092E9008091F000877F8093F000789487
:1018C0000E94800C1092E9008091F0008860809363
:1018D000F000CD2BCF70C093E900FF91EF91DF9125
:1018E000CF91BF91AF919F918F917F916F915F91B8
:1018F0004F913F912F910F900FBE0F901F90189511
:101900001F93CF93DF93CDB7DEB7AA970FB6F894A6
:10191000DEBF0FBECDBFE5EEF1E08091F100819317
:1019200021E0ED3EF207C9F70E94FF078091E80031
:1019300083FF24C18091E5019091E601492F50E099
:101940004A30510508F01AC1FA01EA5AFF4F0C94C7
:101950003422803881F0823809F010C18091E90189
:101960008F708093E9008091EB0085FB882780F9D8
:101970001092E90006C08091E1019091E20191117D
:1019800082609091E800977F9093E8008093F10047
:101990001092F100C8C0282F2D7F09F0EFC08823D6
:1019A00019F0823061F0EAC08091E701813009F0DE
:1019B000E5C0933009F080E08093E2012BC0809174
:1019C000E701811127C08091E9018F7009F4D6C029
:1019D0008093E9002091EB0020FF1CC0933021F49C
:1019E0008091EB00806214C09091EB009061909325
:1019F000EB0021E030E0A90102C0440F551F8A9599
:101A0000E2F74093EA001092EA008091EB008860D0
:101A10008093EB001092E9008091E800877F86C0F8
:101A20008111ACC01091E7011F778091E3008078AD
:101A3000812B8093E3008091E800877F8093E8000A
:101A40000E949D0A8091E80080FFFCCF8091E30016
:101A500080688093E300111102C082E001C083E03E
:101A60008093E4018BC08058823008F087C0809159
:101A7000E7019091E8018C3D53E0950779F583E00B
:101A80008A838AE289834FB7F894DE01139620E0B7
:101A90003EE051E2E32FF0E050935700E49120FF45
:101AA00003C0E295EF703F5FEF708E2F90E0EA3059
:101AB00010F0C79601C0C0968D939D932F5F24317F
:101AC00049F74FBF8091E800877F8093E8006AE282
:101AD00070E0CE0101960E94A90914C0AE014F5FCB
:101AE0005F4F6091E9010E94F208BC01892B09F463
:101AF00045C09091E800977F9093E80089819A8192
:101B00000E94070A8091E8008B778093E80036C036
:101B10008038A1F58091E800877F8093E80080916C
:101B2000E0018093F1008091E8008E778093E800D7
:101B30000E949D0A23C0811121C08091E7019091EC
:101B4000E80199270297D4F48091E800877F809379
:101B5000E8008091E7018093E0010E949D0A809156
:101B6000E001811106C08091E30087FD02C081E0A1
:101B700001C084E08093E4010E94EB078091E800BB
:101B800083FF0AC08091E800877F8093E8008091FE
:101B9000EB0080628093EB00AA960FB6F894DEBF4C
:101BA0000FBECDBFDF91CF911F9108950895CF93C0
:101BB0008091E4018823A1F0C091E900CF70909159
:101BC000EC00892F817090FD80E8C82B1092E9000D
:101BD0008091E80083FD0E94800CCF70C093E900E3
:101BE000CF91089590936901809368010895E091E1
:101BF0006801F0916901309721F00190F081E02DAA
:101C0000099480E00895E0916801F09169013097AE
:101C100021F00280F381E02D09940895E09168019C
:101C2000F0916901309721F00480F581E02D09944D
:101C3000089520916601309167012817390771F0E6
:101C40009093670180936601E0916801F0916901CA
:101C5000309721F00680F781E02D099408952091B6
:101C60006401309165012817390771F0909365017F
:101C700080936401E0916801F0916901309721F04F
:101C80000084F185E02D0994089508950C94450E83
:101C90000E94031A0E94B5030C94C91ACF92DF92D6
:101CA000EF92FF920F931F93CF93DF93CDB7DEB7E1
:101CB0002B970FB6F894DEBF0FBECDBF0E94CD03A9
:101CC0008BE6C82E81E0D82E00E010E0E02E802FB9
:101CD0000E94C304F60141916F01F82EF426B1F47D
:101CE0000F5F1F4F0E30110589F78FEF89838A83AD
:101CF0001B820E940C1A8160782F9D838C834981FE
:101D00005A816B818D810E94F10E40C09091CC016F
:101D100091FF04C08B870E94C9048B8520E030E0CE
:101D20004F2D50E0922FBA01022E02C07595679593
:101D30000A94E2F760FF24C02E83EF8221E030E0B6
:101D4000690102C0CC0CDD1C9A95E2F790E08C2171
:101D50009D21892B09F420E028870E940C1A8160BC
:101D6000782F9A8789874E815F8168858A850E944E
:101D7000F10EF801E559FE4F8081C826C08206C0E9
:101D80002F5F3F4F2630310569F6AACF0E94B01D64
:101D90000E94F70D90916A018917A1F00E94F70D3A
:101DA00080936A012B960FB6F894DEBF0FBECDBFAD
:101DB000DF91CF911F910F91FF90EF90DF90CF9027
:101DC0000C94ED062B960FB6F894DEBF0FBECDBF78
:101DD000DF91CF911F910F91FF90EF90DF90CF9007
:101DE0000895CF93DF93CDB7DEB72B970FB6F89456
:101DF000DEBF0FBECDBF4F83588769877A878B8739
:101E0000DE01119686E0FD0111928A95E9F785E0E1
:101E1000FE01379601900D928A95E1F749815A812A
:101E20006B817C818D819E810E94F4152B960FB66B
:101E3000F894DEBF0FBECDBFDF91CF910895CF9351
:101E4000C82F882309F4C1C0823859F40E94F70DC5
:101E500081FDBBC089E30E9491180E94491989E362
:101E60000CC0833879F40E94F70D80FDAEC083E585
:101E70000E9491180E94491983E50E94D018CF91C1
:101E80000C944919843859F40E94F70D82FD9DC0C5
:101E900087E40E9491180E94491987E4EECF8CEFE5
:101EA0008C0F813A48F48C2F0E94F01F81118DC055
:101EB0008C2F0E949118E3CF80E28C0F883048F479
:101EC000C77081E001C0880FCA95EAF70E94121915
:101ED000D6CF8BE58C0F833078F4C53A29F0C63A1B
:101EE00031F083E890E005C081E890E002C082E82C
:101EF00090E0CF910C94190E88E58C0F833108F097
:101F000064C0C83A39F1C93A41F1CA3A49F1CB3A09
:101F100051F1CC3A59F1CD3A61F1C03B69F1CE3A79
:101F200071F1CF3A79F1C13B81F1C23B89F1C33BF9
:101F300091F1C43B99F1C53BA1F1C63BA9F1C73B67
:101F4000B1F1C83BB9F1C93BC1F1CA3BC9F180E06D
:101F500090E038C082EE90E035C089EE90E032C06B
:101F60008AEE90E02FC085EB90E02CC086EB90E0ED
:101F700029C087EB90E026C08CEC90E023C08DEC6C
:101F800090E020C083E891E01DC08AE891E01AC08B
:101F900082E991E017C084E991E014C081E292E007
:101FA00011C083E292E00EC084E292E00BC085E2B1
:101FB00092E008C086E292E005C087E292E002C0AB
:101FC0008AE292E0CF910C942F0ECF91089588234E
:101FD00009F44BC0823859F40E94F70D81FF45C0C7
:101FE00089E30E9491180E94491989E30CC0833843
:101FF00071F40E94F70D80FF38C083E50E949118AC
:102000000E94491983E50E94D0180C94491984381C
:1020100059F40E94F70D82FF28C087E40E949118AE
:102020000E94491987E4EFCF9CEF980F913A58F33B
:1020300090E2980F983050F4877091E001C0990FAA
:102040008A95EAF7892F0E941819DFCF9BE5980F30
:10205000933020F480E090E00C94190E885A83317C
:1020600020F480E090E00C942F0E0895882321F056
:102070000E9412190C9449190895882321F00E9496
:1020800018190C9449190895BF92CF92DF92EF92DC
:10209000FF920F931F93CF93DF9300D000D000D017
:1020A000CDB7DEB77C0185E0F701DE011196019026
:1020B0000D928A95E1F7F70183819481892B09F4C8
:1020C000DDC2908181818F3F19F49F3F09F4D6C210
:1020D000F7010281258122952F7099838A83898156
:1020E0009A812E830E945018182FB92E0E944F18E3
:1020F0000E941617EB2DE295EF704E2F50E0FA017B
:10210000E05AFF4F2E810C9434228B2D807F9B2D23
:102110009F70F92E882319F0F29480EFF8220023A3
:1021200049F0FF2009F457C28F2D0E9422190E9406
:10213000491951C2812F0E94E70FFF2009F49EC266
:102140008F2D0E94281926960FB6F894DEBF0FBE79
:10215000CDBFDF91CF911F910F91FF90EF90DF9056
:10216000CF90BF900C9449193B2D307F8B2D8F70F1
:10217000303211F08295807F112319F0113021F156
:102180002CC00023B9F0222309F490C1213009F0BA
:102190008DC126960FB6F894DEBF0FBECDBFDF917E
:1021A000CF911F910F91FF90EF90DF90CF90BF9054
:1021B0000C943219222319F0213009F45FC28E8366
:1021C0000E9435198E8186C1002321F0223008F04B
:1021D00055C26CC1211152C27DC1002321F02223BE
:1021E00009F464C1F8C1222309F474C109C28B2D1A
:1021F00086958695837019F08130D1F03FC2002317
:1022000021F0812F9B2D937002C080E090E02696F4
:102210000FB6F894DEBF0FBECDBFDF91CF911F91F7
:102220000F91FF90EF90DF90CF90BF900C94190E1C
:10223000002321F0812F9B2D937002C080E090E05D
:1022400026960FB6F894DEBF0FBECDBFDF91CF91BB
:102250001F910F91FF90EF90DF90CF90BF900C9463
:102260002F0E812F002319F00E94B81C02C00E947B
:10227000201D26960FB6F894DEBF0FBECDBFDF91AE
:10228000CF911F910F91FF90EF90DF90CF90BF9073
:102290000C94A51D8B2D837009F075C00111EEC142
:1022A000812F829586958770880F880F912F9F7058
:1022B000C92ED12CE12CF12C082E04C0CC0CDD1C35
:1022C000EE1CFF1C0A94D2F714FF12C00FE010E0BE
:1022D00020E030E004C0000F111F221F331F8A9539
:1022E000D2F7C901B801609570958095909503C0AB
:1022F00060E070E0CB014B2D46954695437042302F
:10230000C1F060F56C297D298E299F29413051F15A
:1023100026960FB6F894DEBF0FBECDBFDF91CF91EA
:102320001F910F91FF90EF90DF90CF90BF900C9492
:102330003D176C297D298E299F2926960FB6F89482
:10234000DEBF0FBECDBFDF91CF911F910F91FF90E8
:10235000EF90DF90CF90BF900C9459170E943D17DB
:10236000C701B60126960FB6F894DEBF0FBECDBFEB
:10237000DF91CF911F910F91FF90EF90DF90CF9061
:10238000BF900C942117002319F08B2D817001C090
:102390008695882309F472C1812F8295869587706E
:1023A000880F880F912F9F70C92ED12CE12CF12C12
:1023B000082E04C0CC0CDD1CEE1CFF1C0A94D2F7C6
:1023C00014FF12C00FE010E020E030E004C0000F66
:1023D000111F221F331F8A95D2F7C901B8016095DA
:1023E00070958095909503C060E070E0CB014B2D17
:1023F0004695469543704230C1F060F56C297D29C1
:102400008E299F29413051F126960FB6F894DEBFF0
:102410000FBECDBFDF91CF911F910F91FF90EF9035
:10242000DF90CF90BF900C9417186C297D298E29CE
:102430009F2926960FB6F894DEBF0FBECDBFDF9161
:10244000CF911F910F91FF90EF90DF90CF90BF90B1
:102450000C9433180E941718C701B60126960FB6C0
:10246000F894DEBF0FBECDBFDF91CF911F910F91CA
:10247000FF90EF90DF90CF90BF900C94FB17103F30
:10248000D1F118F4103E50F4A1C0123F09F463C01A
:1024900008F44CC0133F09F473C098C01F708B2D13
:1024A0008F710023A1F00E949417812F26960FB6FA
:1024B000F894DEBF0FBECDBFDF91CF911F910F917A
:1024C000FF90EF90DF90CF90BF900C9436100E9459
:1024D000B517812F26960FB6F894DEBF0FBECDBF7D
:1024E000DF91CF911F910F91FF90EF90DF90CF90F0
:1024F000BF900C943D100023A9F02111BFC08B2D7B
:102500008F7126960FB6F894DEBF0FBECDBFDF9158
:10251000CF911F910F91FF90EF90DF90CF90BF90E0
:102520000C94DA17223008F0A9C0E9CF0023A9F0F3
:102530008B2D8F7126960FB6F894DEBF0FBECDBFE0
:10254000DF91CF911F910F91FF90EF90DF90CF908F
:10255000BF900C949417002359F38B2D8F712696FE
:102560000FB6F894DEBF0FBECDBFDF91CF911F91A4
:102570000F91FF90EF90DF90CF90BF900C94B51724
:10258000002399F08B2D8F7126960FB6F894DEBF3D
:102590000FBECDBFDF91CF911F910F91FF90EF90B4
:1025A000DF90CF90BF900C947F1726960FB6F894CB
:1025B000DEBF0FBECDBFDF91CF911F910F91FF9076
:1025C000EF90DF90CF90BF900C9475170023A9F087
:1025D000222309F4ADCF812F26960FB6F894DEBFE3
:1025E0000FBECDBFDF91CF911F910F91FF90EF9064
:1025F000DF90CF90BF900C941F0F222309F4ADCF32
:10260000812F26960FB6F894DEBF0FBECDBFDF91A7
:10261000CF911F910F91FF90EF90DF90CF90BF90DF
:102620000C94E70F4B2D4F70612FC7010E94580289
:1026300026960FB6F894DEBF0FBECDBFDF91CF91C7
:102640001F910F91FF90EF90DF90CF90BF900C946F
:1026500099164B2D4F70612FC70126960FB6F8942F
:10266000DEBF0FBECDBFDF91CF911F910F91FF90C5
:10267000EF90DF90CF90BF900C948A0526960FB60E
:10268000F894DEBF0FBECDBFDF91CF911F910F91A8
:10269000FF90EF90DF90CF90BF9008950E942F1988
:1026A0000E9404190E9449190E94551E0E94A51DEE
:1026B00080E090E00E94190E80E090E00C942F0ED4
:1026C0000E941F190C944E130E945018292F229516
:1026D0002F702C3030F42A3048F42250223078F415
:1026E00005C02C3041F02F3031F009C0803E48F059
:1026F000803F29F406C093FB882780F9089580E085
:10270000089581E00895CF93DF9300D000D01F9209
:10271000CDB7DEB70F900F900F900F900F90DF9115
:10272000CF910895CF93DF9300D000D000D0CDB7E4
:10273000DEB726960FB6F894DEBF0FBECDBFDF9191
:10274000CF9108951F93CF93DF93C091790116E045
:1027500080917A01C81799F0D0E01C9FF0011D9F6D
:10276000F00D1124E558FE4F408151816281738143
:10277000848195810E9492132196C770E9CFDF91E1
:10278000CF911F9108954091AB015091AC016091A0
:10279000AD017091AE018091AF019091B0010C94A8
:1027A00092138091B00182958F7009F054C080918E
:1027B000AD01882309F44FC080917901A0917A017D
:1027C0004091AE015091AF016091AB017091AC01AD
:1027D000B6E08A1709F43FC090E041155105C1F1F8
:1027E0007F3F11F46F3FA1F1B89FF001B99FF00D49
:1027F0001124E558FE4F218127132AC0208126137A
:1028000027C02281211124C0238134812417350758
:1028100010F421503109241B350B283C3105C0F43C
:102820002091B0012F7020612093B00126E0289FF5
:10283000F001299FF00D1124E058FE4F80818F7028
:10284000806180838BEA91E00E9444100C94A21373
:1028500001968770BECF0895CF92DF92EF92FF92DC
:102860000F931F93CF93DF93CDB7DEB762970FB669
:10287000F894DEBF0FBECDBF8C0185E0F801DE010C
:102880001D9601900D928A95E1F7D8014C91119611
:102890005C91119712966C918091AE019091AF016D
:1028A000009709F475C13091AB017091AC017F3F85
:1028B00019F43F3F09F46CC1F801C380D480E09063
:1028C000AD01EE2009F4BEC02091B001C816D906B2
:1028D00028F0D601A81BB90BCD0104C080959095B6
:1028E0008C0D9D1DFF24F394883C910578F0F12C0C
:1028F000207F09F0C4C07C2DD98AC88A89890E94AA
:1029000083138BEA91E00E944410AFC0822F807F36
:1029100009F045C0571313C0431311C061110FC014
:102920002F7020612093B0010E94C3138BEA91E0C5
:102930000E9444108091B001F80185832EC0CD28FB
:1029400019F15F3F11F44F3FF9F0F62E61111CC0F1
:102950008091790120917A0136E0821709F45BC0F9
:1029600090E0389FF001399FF00D1124E558FE4F9B
:102970007181571306C07081471303C072817111B2
:1029800003C001968770E9CFF62E662309F41CC1B7
:102990008091B00181608093B001F12C15C1571373
:1029A00009C0431307C0611105C08091B001F8014F
:1029B0008583C8C04D875E878D859E856A8B0E9402
:1029C00064136A898823D1F16623C1F12091B00193
:1029D000822F82958F7090E0029774F08091AB0106
:1029E0009091AC0198878F831986DB86CA862C87E5
:1029F000CE0107960E94441086E0F801ABEAB1E0F0
:102A000001900D928A95E1F70E94D1130E94C313A1
:102A1000FF24F394D9C04D875E878D859E850E94E3
:102A20005018292F22952F70223008F0C1C09F70B6
:102A300009F0BBC0805E883008F4C6C0C8010E949F
:102A40004410E6CFC816D90608F453C0F601E81BB7
:102A5000F90BCF01883C910508F450C0F12C7C2D76
:102A6000D98AC88A89890E948313EBEAF1E086E05B
:102A7000DF011D928A95E9F70E94C313A5C0571381
:102A800014C0431312C0611110C08091B001F8014D
:102A90008583C8010E94441086E0EBEAF1E0DF0183
:102AA0001D928A95E9F7FE2C8FC04D875E878D8534
:102AB0009E856A8B0E9464136A89882309F4BECFBD
:102AC000662309F4BBCF2091B001822F82958F70CD
:102AD00090E002970CF490CF8091AB019091AC0103
:102AE0009A8389831B82DD82CC822E83CE0101965C
:102AF00081CF809590958C0D9D1DACCFF62E6623D1
:102B000009F49CCF571333C0431331C02091B00157
:102B100020FD24C0822F82958F70482F50E04115F0
:102B20005105E1F0D80115962C9315974F305105BA
:102B300049F08F5F982F9295907F822F8F70892B0D
:102B400015968C93C8010E94441086E0F801ABEA08
:102B5000B1E001900D928A95E1F78ECF86E0F80101
:102B6000ABEAB1E001900D928A95E1F72DC04D8757
:102B70005E878D859E850E94641381113DCF809173
:102B8000B00181608093B001C8010E9444101CC054
:102B9000662309F453CF4D875E878D859E850E94FD
:102BA0006413882309F44ACF27CF811143CF0CC087
:102BB000243008F043CF9F7009F43CCFD80115961C
:102BC0009C91907F09F036CF8F2D62960FB6F894C6
:102BD000DEBF0FBECDBFDF91CF911F910F91FF9050
:102BE000EF90DF90CF9008951F93CF93DF93CDB7F1
:102BF000DEB72C970FB6F894DEBF0FBECDBF4F8364
:102C0000588769877A878B879C87CE0107960E94B1
:102C10002C14882371F08A859B85892B09F441C087
:102C200088858F3F09F065C08F818F3F09F061C0B3
:102C300038C086E0FE013796DE01119601900D92B4
:102C40008A95E1F76A857B856115710551F1FF81F0
:102C5000E885EF3F11F4FF3F21F120917A0130E048
:102C6000C9010196877099274091790150E0841736
:102C7000950709F447C0F983EA837D836C8396E066
:102C8000929FD001939FB00D1124A558BE4FFE0115
:102C9000319601900D929A95E1F780937A010E9406
:102CA000A21316E08091790190917A018917B9F108
:102CB000189FC001112485589E4F0E942C14882310
:102CC00071F1E09179011E9FF0011124E558FE4F4A
:102CD0004081518162817381848195810E94921328
:102CE0008091790190E0019687709927809379010E
:102CF000D9CF4F81588569857A858B859C850E94BF
:102D00009213CFCF0E94601310927A011092790132
:102D1000EBEAF1E086E0DF011D928A95E9F72C9657
:102D20000FB6F894DEBF0FBECDBFDF91CF911F91DC
:102D30000895EF92FF920F931F93CF93DF938C012F
:102D4000892B09F46CC0F12CEE24E394E801219660
:102D5000F8018491843740F4843008F051C0813008
:102D600081F0823019F15BC0853709F444C0A8F1C5
:102D70009CE7980F903708F052C08F770E94E70FBA
:102D800041C00E5F1F4FFE01849190E2980F983072
:102D900050F48770FE2D01C0FF0F8A95EAF78F2F40
:102DA0000E94221914C00E941F0F2DC00E5F1F4FDA
:102DB000FE01849190E2980F983060F48770FE2DA8
:102DC00001C0FF0F8A95EAF78F2F0E9428190E94F1
:102DD000491919C00E94E70F16C00E5F1F4FFE0170
:102DE000C491CC2381F08FE99FE00197F1F700C0F7
:102DF0000000C150F6CF0E5F1F4FFE01F49003C0DC
:102E00000E941F0F8E018F2D882309F49FCFEFE9B9
:102E1000FFE03197F1F700C000008150F5CFDF915E
:102E2000CF911F910F91FF90EF90089508956093B7
:102E3000B5017093B6018093B7019093B8010C94DB
:102E40004E130F931F930091B5011091B60120917D
:102E5000B7013091B801DC01CB01802B912BA22B63
:102E6000B32B8093B5019093B601A093B701B093B3
:102E7000B8011F910F910C944E130F931F93009163
:102E8000B5011091B6012091B7013091B801DC0174
:102E9000CB0180239123A223B3238093B501909388
:102EA000B601A093B701B093B8011F910F910C9494
:102EB0004E130F931F930091B5011091B60120910D
:102EC000B7013091B801DC01CB0180279127A227FF
:102ED000B3278093B5019093B601A093B701B09347
:102EE000B8011F910F910C944E131092B1011092E2
:102EF000B2011092B3011092B4010C944E1341E050
:102F000050E060E070E004C0440F551F661F771F5B
:102F10008A95D2F74093B1015093B2016093B30107
:102F20007093B4010C944E1341E050E060E070E007
:102F300004C0440F551F661F771F8A95D2F78091F2
:102F4000B1019091B201A091B301B091B401482BAD
:102F5000592B6A2B7B2B4093B1015093B2016093A4
:102F6000B3017093B4010C944E1341E050E060E063
:102F700070E004C0440F551F661F771F8A95D2F773
:102F800040955095609570958091B1019091B201F6
:102F9000A091B301B091B401482359236A237B2344
:102FA0004093B1015093B2016093B3017093B401A7
:102FB0000C944E1341E050E060E070E004C0440F18
:102FC000551F661F771F8A95D2F78091B1019091A6
:102FD000B201A091B301B091B401482759276A27E3
:102FE0007B274093B1015093B2016093B30170937A
:102FF000B4010C944E130F931F930091B1011091E3
:10300000B2012091B3013091B401DC01CB01802BDE
:10301000912BA22BB32B8093B1019093B201A0937B
:10302000B301B093B4011F910F910C944E130F9301
:103030001F930091B1011091B2012091B301309121
:10304000B401DC01CB0180239123A223B32380931D
:10305000B1019093B201A093B301B093B4011F9159
:103060000F910C944E130F931F930091B101109187
:10307000B2012091B3013091B401DC01CB01802772
:103080009127A227B3278093B1019093B201A09317
:10309000B301B093B4011F910F910C944E13089596
:1030A000CF92DF92EF92FF920F931F93CF93DF9314
:1030B0008C01C090B101D090B201E090B301F090CA
:1030C000B4018091B5019091B601A091B701B09182
:1030D000B801C82AD92AEA2AFB2ACFE1D0E0D701D1
:1030E000C6010C2E04C0B695A795979587950A94AE
:1030F000D2F780FF07C0B8018C2F0E94AE05813047
:10310000910531F4219758F7B80180E00E94AE058F
:10311000DF91CF911F910F91FF90EF90DF90CF90B3
:10312000089590910C019923F1F090910D0199234C
:10313000D1F0982F9695969596959F3080F5E091D1
:103140000E01F0910F01E90FF11D877021E030E0D1
:10315000A90102C0440F551F8A95E2F7CA01918167
:10316000892B8183089520910E0130910F01F9017F
:1031700032969FEF40E05191851789F09F3F19F4F7
:10318000511101C0942F4F5F4E30A9F79F3F39F086
:10319000F901E90FF11D97FDFA95828308950895CD
:1031A00090910C019923F9F090910D019923D9F098
:1031B000982F9695969596959F3028F5E0910E015B
:1031C000F0910F01E90FF11D877021E030E0A901B6
:1031D00002C0440F551F8A95E2F7CA01809591817C
:1031E00089238183089520910E0130910F01F90107
:1031F0003296205F3F4F9081891301C01082319633
:10320000E217F307C1F7089581E090E0E0910E0125
:10321000F0910F01E80FF91F10820196803191059E
:10322000A9F708959091CB01892B8093CB01089544
:1032300080959091CB0189238093CB0108951092C2
:10324000CB0108959091CA01892B8093CA010895FA
:1032500080959091CA0189238093CA0108951092A4
:10326000CA0108958093B90108951092B901089593
:1032700080910E0190910F01FC0131969C01205F1D
:103280003F4F80E0919191118F5FE217F307D1F7E3
:103290000895E0910E01F0910F018091CB018083A0
:1032A000E0910E01F0910F0190818091CA01892B6C
:1032B00080838091B901882361F0E0910E01F09143
:1032C0000F019081892B80830E94381981111092FF
:1032D000B90180910E0190910F010C94030ECF92D1
:1032E000DF92EF92FF926C01EE24FF24C114D1040F
:1032F000E104F10421F0C701B60120E101C020E0A2
:10330000C72ED82EE92EFF24C114D104E104F10404
:1033100019F0285FC701B6016B017C0154E0F694F7
:10332000E794D794C7945A95D1F7C114D104E10416
:10333000F10419F02C5FC701B6016B017C0142E07A
:10334000F694E794D794C7944A95D1F7C114D10461
:10335000E104F10419F02E5FC701B601DC01CB01D5
:10336000B695A79597958795892B8A2B8B2B09F076
:103370002F5F822FFF90EF90DF90CF900895809184
:10338000E401843011F120E488E190E00FB6F89474
:10339000A895809360000FBE2093600083B7817F63
:1033A000846083BF83B7816083BF7894889583B737
:1033B0008E7F83BF0FB6F894A895809160008861D6
:1033C00080936000109260000FBE089508950C94E1
:1033D000E619CF930E94E7190E94CD030E94E619D7
:1033E000C0E08C2F0E94C304811104C0CF5FCE3097
:1033F000C1F701C081E0CF9108950E9460130E943F
:10340000F70D0C94ED0682E084BD93E095BD9AEF34
:1034100097BD80936E0008952FB7F8948091CD01E9
:103420009091CE01A091CF01B091D0012FBF08950E
:10343000CF92DF92EF92FF920F931F932FB7F894E2
:103440004091CD015091CE016091CF017091D0019A
:103450002FBF6A017B01EE24FF248C0120E030E0C5
:10346000C016D106E206F30610F4415051099A0144
:10347000281B390BC9011F910F91FF90EF90DF902E
:10348000CF9008951F920F920FB60F9211248F9331
:103490009F93AF93BF938091CD019091CE01A09166
:1034A000CF01B091D0010196A11DB11D8093CD0136
:1034B0009093CE01A093CF01B093D001BF91AF9173
:1034C0009F918F910F900FBE0F901F9018950E94A3
:1034D000EF0AF8942FEF87EA91E621508040904060
:1034E000E1F700C0000087E090EBDC018093ED0184
:1034F0009093EE01A093EF01B093F0019CE088E17E
:103500000FB6F894A895809360000FBE909360006A
:10351000FFCFEF92FF920F931F93CF93DF93D82F9C
:10352000C0E08C2F0E94C30400E010E0E82EF12CD4
:10353000C701002E02C0959587950A94E2F780FD99
:1035400006C00F5F1F4F0630110591F709C0602FAD
:103550007C2F80E00E948B058D13F3CF81E004C0A7
:10356000CF5FCE30F1F680E0DF91CF911F910F91C8
:10357000FF90EF900895CF93C82F8CE20E94891A94
:10358000882321F08C2FCF910C94891A80E0CF9161
:103590000895CF930E94101C811102C00E94F61B57
:1035A000C5E6C15049F00E94CD038FE39CE9019725
:1035B000F1F700C00000F5CF89E20E94BB1A81112B
:1035C00013C18AE20E94BB1A81110E94F61B85E09A
:1035D0000E94BB1A81110E94671A0E941B1C8093D3
:1035E000CC0187E00E94BB1A8823A9F18BE10E94DD
:1035F000BB1A882351F08091CC0181FB222720F94E
:1036000091E0922790FB81F90EC08EE00E94BB1AD8
:10361000882361F08091CC0182FB222720F991E080
:10362000922790FB82F98093CC0115C080E10E9423
:10363000BB1A9091CC01882341F093FB222720F9FB
:1036400081E0822780FB93F904C0892F809580FB5D
:1036500090F99093CC018091CC010E941F1C0E9494
:103660002D1C8093DE0180EE0E94BB1A882341F05E
:103670008091DE01982F909590FB80F98093DE0178
:1036800089E30E94BB1A882359F08091DE0181FBF7
:10369000222720F991E0922790FB81F98093DE01A7
:1036A00082EE0E94BB1A882359F08091DE0182FBD2
:1036B000222720F991E0922790FB82F98093DE0186
:1036C00086EE0E94BB1A882359F08091DE0183FBAD
:1036D000222720F991E0922790FB83F98093DE0165
:1036E00083EE0E94BB1A882359F08091DE0184FB8F
:1036F000222720F991E0922790FB84F98093DE0144
:1037000085E30E94BB1A882359F08091DE0185FB76
:10371000222720F991E0922790FB85F98093DE0122
:1037200081E30E94BB1A882359F08091DE0186FB59
:10373000222720F991E0922790FB86F98093DE0101
:1037400081E10E94BB1A882359F08091DE0187FB3A
:10375000222720F991E0922790FB87F98093DE01E0
:103760008091DE010E94311C8091DE0187FB882759
:1037700080F980930D0187E20E94BB1AC82F8EE169
:103780000E94BB1A8111C2608FE10E94BB1A811195
:10379000C46080E20E94BB1A8111C86081E20E946D
:1037A000BB1A8111C06182E20E94BB1A8111C06202
:1037B00083E20E94BB1A8111C06484E20E94BB1A9A
:1037C000882311F0C06802C0CC2329F08C2F0E94FE
:1037D000281C6C2F03C00E94241C682F70E080E01E
:1037E00090E0CF910C941717CF9108956DEE7EEF76
:1037F00080E090E00E946A2260E082E090E00E9417
:103800005C2260E083E090E00E945C2260E084E063
:1038100090E00E945C2260E085E090E00C945C22E5
:1038200080E090E00E94562221E08D3E9E4F09F0FC
:1038300020E0822F089582E090E00C944E22682FC1
:1038400082E090E00C945C2283E090E00C944E22A5
:10385000682F83E090E00C945C2284E090E00C946C
:103860004E22682F84E090E00C945C228091D3017A
:1038700080FF0BC06091130185E0689FB0011124A7
:1038800075956795759567952BC081FF09C0609107
:10389000130185E0689FB00111247595679520C0DC
:1038A00082FF07C06091130185E0689FB001112479
:1038B00017C09091D4019923D1F06091120196170D
:1038C00088F72091130185E0289F90011124929F91
:1038D000A001939F500D112470E0CA010E94202284
:1038E0006038710540F46115710519F406C065E092
:1038F00070E0862F08958FE7089581E00895809104
:10390000D30180FF08C06091110170E07595679543
:103910007595679521C081FF06C06091110170E027
:103920007595679519C082FF04C06091110170E020
:1039300010C09091D401992399F0609110019617CD
:10394000A0F780911101899FC001112470E00E94AD
:1039500020226038710540F46115710519F406C024
:1039600061E070E0862F08958FE7089581E0089563
:10397000803F21F40E94361C819504C0813F29F4C8
:103980000E94361C8093D7010895823F21F40E9443
:10399000361C819504C0833F29F40E94361C809315
:1039A000D6010895893F19F40E947F1C05C08A3F03
:1039B00031F40E947F1C81958093D80108958B3F3C
:1039C00021F40E947F1C819504C08C3F29F40E9441
:1039D0007F1C8093D9010895843F21F48091D50103
:1039E000816017C0853F21F48091D501826011C0AC
:1039F000863F21F48091D50184600BC0873F21F47C
:103A00008091D501886005C0883F31F48091D5014F
:103A100080618093D50108958D3F21F48091D30179
:103A200081600BC08E3F21F48091D301826005C07C
:103A30008F3F29F48091D30184608093D30108954E
:103A4000803F39F48091D70187FF6CC01092D70175
:103A500069C0813F29F48091D7011816BCF362C078
:103A60009091D601823F29F497FF5CC01092D60155
:103A700059C0833F19F41916CCF354C0893F41F45F
:103A80008091D80118160CF04DC01092D8014AC090
:103A90008A3F29F48091D80187FF44C0F6CF8B3F3D
:103AA00039F48091D90187FF3DC01092D9013AC005
:103AB0008C3F29F48091D9011816BCF333C0843FA0
:103AC00021F48091D5018E7F17C0853F21F480912C
:103AD000D5018D7F11C0863F21F48091D5018B7F68
:103AE0000BC0873F21F48091D501877F05C0883FB7
:103AF00031F48091D5018F7E8093D50113C08D3F25
:103B000021F48091D3018E7F0BC08E3F21F48091F0
:103B1000D3018D7F05C08F3F29F48091D3018B7F26
:103B20008093D3018091D60181110EC08091D7017D
:103B300081110AC08091D801811106C08091D901FC
:103B4000811102C01092D401089585ED91E00E9488
:103B50000E0E0E940C1A9093D2018093D101089509
:103B60001F93CF93DF938091D1019091D2010E9456
:103B7000181AAC019091D401992321F020911401DD
:103B800030E006C0209115018AE0289F90011124A1
:103B90004217530708F485C08091D601C091D70120
:103BA000D091D8011091D901811107C0C11175C000
:103BB000D11173C0111171C074C09F3F19F09F5F84
:103BC0009093D401181624F40E94361C8093D601D9
:103BD0008091D60187FF05C00E94361C8195809395
:103BE000D6011C1624F40E94361C8093D7018091C4
:103BF000D70187FF05C00E94361C81958093D701AD
:103C00006091D601662331F1C091D701CC2311F127
:103C1000062E000C770B880B990B0E94272123E3BB
:103C200033E343E35FE30E948B210E94EF20609324
:103C3000D6016C2FCC0F770B880B990B0E94272194
:103C400023E333E343E35FE30E948B210E94EF20F1
:103C50006093D7011D1624F40E947F1C8093D80125
:103C60008091D80187FF05C00E947F1C81958093B9
:103C7000D801111624F40E947F1C8093D9018091F1
:103C8000D90187FF05C00E947F1C81958093D901CF
:103C9000DF91CF911F910C94A51D9F3F09F08FCF0D
:103CA000A0CFDF91CF911F910895E5EDF1E085E080
:103CB000DF011D928A95E9F71092D4011092D30189
:103CC0000895833081F128F4813059F08230D1F0A9
:103CD0000895853009F449C0B8F1863009F456C01A
:103CE000089580911501262F30E0280F311D2F3FB8
:103CF000310524F4680F6093150108958FEF8093C8
:103D00001501089580911401262F30E0280F311DF0
:103D10002F3F310524F4680F6093140108958FEF4D
:103D200080931401089580911301262F30E0280F0D
:103D3000311D2F3F310524F4680F6093130108955E
:103D40008FEF80931301089580911201262F30E0A8
:103D5000280F311D2F3F310524F4680F60931201A5
:103D600008958FEF80931201089580911101262FFD
:103D700030E0280F311D2F3F310524F4680F609388
:103D8000110108958FEF8093110108958091100122
:103D9000262F30E0280F311D2F3F310524F4680F06
:103DA0006093100108958FEF809310010895833080
:103DB00011F128F4813049F0823091F00895853076
:103DC00081F120F18630C1F10895809115016817C5
:103DD00020F4861B80931501089510921501089513
:103DE00080911401681720F4861B809314010895B4
:103DF00010921401089580911301681720F4861B16
:103E00008093130108951092130108958091120177
:103E1000681720F4861B80931201089510921201F6
:103E2000089580911101681720F4861B8093110179
:103E3000089510921101089580911001681720F4DF
:103E4000861B8093100108951092100108950F931E
:103E50001F938D3109F46BC008F03FC08E3009F418
:103E60007DC0C0F4873009F46EC068F4863009F074
:103E7000AFC08091CC01817F8E7F8093CC0181E0A7
:103E80008093DB01A6C0883009F458C08B3009F458
:103E90009BC09EC0863109F497C078F4803109F444
:103EA00070C0813109F094C00E94601390910D019F
:103EB00081E0892780930D0187C0893109F484C08E
:103EC0008B3109F085C08091CC0181FB222720F93C
:103ED00091E0922790FB81F94AC0853309F45BC0D9
:103EE00048F4873209F457C008F45AC0893209F4FB
:103EF00052C06EC0833438F48A3308F067C0883308
:103F000009F462C065C0833409F445C0883409F0FF
:103F10005FC00E9460130FEF13ED20E301501040CB
:103F20002040E1F700C000000E94671A4DC00E94C7
:103F3000A9200E94F70D0E94ED0646C00E941B1C9E
:103F40000E942D1C41C09091CC01892F817090FF5F
:103F500012C0917F9E7F9093CC013BC08091CC0199
:103F600082FB222720F991E0922790FB82F980932F
:103F7000CC01992349F18091CC0181608093CC01DF
:103F800023C08091CC0183FB222720F991E0922766
:103F900090FB83F9ECCF61E070E080E090E010C02E
:103FA0008D5141E050E060E070E08A019B0104C067
:103FB000000F111F221F331F8A95D2F7C901B801C4
:103FC0000E9417170E94601381E003C08953E9CF54
:103FD00080E01F910F91089580E008950C94EC1FEC
:103FE000CF93C82F8091DB01813079F018F08230B7
:103FF000E9F187C0E0910E01F0910F0180818131DC
:1040000069F0823209F07FC009C0E0910E01F091A1
:104010000F018081813111F0823261F48C2F0E9476
:10402000EE1F811104C08C2F0E94271F1DC081E04C
:1040300090E01AC08C2F0E94EC1F811114C0C43173
:1040400079F048F4CB3079F0C03109F060C082E0FB
:104050008093DB0108C0C93219F0C83321F057C082
:104060001092DB0154C081E0817053C0C93289F1E4
:1040700018F5C43171F1A8F4C73009F046C08AE0E0
:104080008093150194E19093140193E090931301B0
:104090008093120188E08093110188E280931001DF
:1040A00034C0CE51C63088F5EC2FF0E0E65DFE4F0F
:1040B00080818093DA0129C0CE34E9F020F4CB343A
:1040C00021F56AE013C0C13579F0C235F1F461E041
:1040D0000DC08091DA01882319F01092DA0115C021
:1040E00081E08093DB0115C061E006C08091DA01B8
:1040F0000E94611E0AC06AE08091DA010E94D71E08
:1041000004C01092DB0180E004C081E002C080E0C6
:10411000ABCFCF910895E1E8F0E0808188608083A3
:104120008081816080838FB7F89493E090938900B9
:1041300090ED909388008FBF0895EFE6F0E08081C6
:10414000826080830895EFE6F0E080818D7F808338
:104150000895EFE6F0E0908182E08927808308955A
:104160001F920F920FB60F9211242F933F934F93EC
:104170005F936F937F938F939F93AF93BF93EF93CF
:10418000FF938091DC019091DD0101969093DD0118
:104190008093DC01811103C082E00E94ED06E09172
:1041A000DD01E695E695F0E0E252FC4FE491809166
:1041B000DC018E1303C080E00E94ED06FF91EF91B9
:1041C000BF91AF919F918F917F916F915F914F912F
:1041D0003F912F910F900FBE0F901F9018950E9446
:1041E000F6206894B1110C94852108950E946A21EB
:1041F00088F09F5798F0B92F9927B751B0F0E1F0A8
:10420000660F771F881F991F1AF0BA95C9F714C057
:10421000B13091F00E948421B1E008950C94842182
:10422000672F782F8827B85F39F0B93FCCF3869590
:1042300077956795B395D9F73EF4909580957095ED
:1042400061957F4F8F4F9F4F0895E89409C097FB6A
:104250003EF490958095709561957F4F8F4F9F4F5D
:104260009923A9F0F92F96E9BB279395F6958795A1
:1042700077956795B795F111F8CFFAF4BB0F11F464
:1042800060FF1BC06F5F7F4F8F4F9F4F16C088230B
:1042900011F096E911C0772321F09EE8872F762F41
:1042A00005C0662371F096E8862F70E060E02AF082
:1042B0009A95660F771F881FDAF7880F969587956E
:1042C00097F9089557FD9058440F551F59F05F3FD7
:1042D00071F04795880F97FB991F61F09F3F79F028
:1042E00087950895121613061406551FF2CF4695AA
:1042F000F1DF08C0161617061806991FF1CF86952C
:104300007105610508940895E894BB27662777270F
:10431000CB0197F908950E949E210C940F220E94D0
:10432000012238F00E94082220F0952311F00C940D
:10433000F8210C94FE2111240C9485210E94622105
:1043400070F3959FC1F3950F50E0551F629FF001E8
:10435000729FBB27F00DB11D639FAA27F00DB11D01
:10436000AA1F649F6627B00DA11D661F829F22278A
:10437000B00DA11D621F739FB00DA11D621F839F11
:10438000A00D611D221F749F3327A00D611D231FE7
:10439000849F600D211D822F762F6A2F11249F5735
:1043A00050409AF0F1F088234AF0EE0FFF1FBB1F38
:1043B000661F771F881F91505040A9F79E3F5105F7
:1043C00080F00C94F8210C9485215F3FE4F3983E33
:1043D000D4F3869577956795B795F795E7959F5FA1
:1043E000C1F7FE2B880F911D9695879597F9089533
:1043F00097F99F6780E870E060E008959FEF80EC98
:10440000089500240A94161617061806090608953A
:1044100000240A9412161306140605060895092EA0
:104420000394000C11F4882352F0BB0F40F4BF2B0F
:1044300011F460FF04C06F5F7F4F8F4F9F4F08954F
:1044400097FB072E16F4009407D077FD09D00E9441
:104450003A2207FC05D03EF4909581959F4F089530
:10446000709561957F4F0895EE0FFF1F0590F491B1
:10447000E02D0994AA1BBB1B51E107C0AA1FBB1F5B
:10448000A617B70710F0A61BB70B881F991F5A95E0
:10449000A9F780959095BC01CD010895F999FECFBB
:1044A00092BD81BDF89A992780B50895A8E1B0E042
:1044B00042E050E00C947122262FF999FECF1FBAEA
:1044C00092BD81BD20BD0FB6F894FA9AF99A0FBE3D
:1044D000019608950E945C22272F0C945D22DC0136
:1044E000CB01FC01F999FECF06C0F2BDE1BDF89AFF
:1044F000319600B40D9241505040B8F70895F894A9
:02450000FFCFEB
:104502002002EE067E0759072507F1060101BA01CE
:1045120028080A03140A3F4D36399F0352031C032D
:10452200E30276028F02A802C10201020304050619
:04453200070809006D
:00000001FF
